:1000000000308A0004280000FF238316900000308F
:100010008A00B428A101A201A001A3014308031D85
:100020001428420803192E281030C4000310C00DF4
:10003000C10DA00DA30D43082302031D2128420872
:100040002002031C2A284208A002031CA303430821
:10005000A3020314A10DA20DC40B1628000024292D
:100060001030A000A301BE01BB0CBA0C031C3E283B
:100070003C08A3070318BE0A3D08BE07BE0CA30C2C
:10008000A20CA10CA00B342857298030BC00BB0166
:10009000BA013A080F3C031C652838083B05BD002F
:1000A00039083C05BE003B083D02031D60283C08A2
:1000B0003E02031D60283B08A1003C08A2006828FE
:1000C0000310BC0CBB0CBA0A49280030A100A200E6
:1000D0009829831605118312051183168510831242
:1000E0008510BC013C080F3C031C96283A080039D7
:1000F000A0003B088039A3002008230403198528A9
:10010000831605108312051489288316051083129F
:1001100005100310BA0DBB0D8316051183120515CA
:100120008316051183120511BC0A722883168510E7
:10013000831285148316851083128510003438309D
:10014000840000080319B3280130A100A001A00B0E
:10015000A728A10BA6284A30A000A00BAD280000BC
:100160000000800BA428003484011F30830583160F
:100170001F08F03907389F00073083129F0083164D
:100180001F08F03908389F001F08F0399F001F082A
:100190000F3930389F0083121F080C3981389F00B7
:1001A0000C30A1001F08C33921049F00831685115C
:1001B000831285158316851283128516A7012F08D1
:1001C000B1002E08B0002D08AF002C08AE002B089F
:1001D000AD002A08AC002908AB002808AA009F142B
:1001E0009F18F02883161E088312A8001E08A90075
:1001F0002A082807B8002908B9000318B90A2B08EB
:10020000B9072C083807BA003908BB000318BB0A25
:100210002D08BB072E083A07BC003B08BD00031899
:10022000BD0A2F08BD0730083C07BE003D08BF00CF
:100230000318BF0A3108BF073F08C1003E08C000CD
:10024000C3010530C2000A282208B3002108B20009
:10025000831685150030831285190130013C031D7A
:100260005B29B308031D38293208D23C03183C2906
:10027000B301D230B2004629B308031D4629320823
:10028000273C031C4629B3012830B2002830320233
:10029000B8003308B9000030031C0130B902390836
:1002A000BB003808BA00BD010630BC003028220867
:1002B000B3002108B200B501B401A60126080F3C25
:1002C000031C8429B208031D6829B3080319822975
:1002D0000310340DB800350DB90038080138B400EA
:1002E0003908B500B308031D79293208403C0318CA
:1002F00080294030B2020030031C0130B302822951
:10030000B301B201A60A5E29A7080319912937088B
:100310003502031C9C29031D912934083602031859
:100320009C296430A7003508B9003408B800452876
:100330002208B7002108B60034083604B800350892
:100340003704B900BB003808BA0069200230B80091
:100350009F20BB01BA0169200830B8009F20831696
:10036000851600308312851A0130003A031DB92921
:06037000A703DF28630073
:02400E0004317B
:00000001FF
